:100000005026002055010000510100005101000060
:1000100000000000000000000000000000000000E0
:10002000000000000000000000000000510100007E
:10003000000000000000000051010000510100001C
:100040005101000051010000510100005101000068
:10005000510100005101000051010000F9100000A1
:100060005101000051010000510100005101000048
:1000700051010000000000000000000051010000DC
:100080005101000051010000510100005101000028
:1000900051010000000000000000000051010000BC
:1000A0005101000051010000510100005101000008
:1000B0000000000010B5064C2378002B07D1054B3B
:1000C000002B02D0044800E000BF0123237010BDC4
:1000D000680000200000000034260000044B10B52A
:1000E000002B03D00349044800E000BF10BDC04608
:1000F000000000006C00002034260000024B034A80
:100100005A6005221A60704710E000E0FFFFFF0010
:1001100070B580250B0E0C4A0C4CD8B26D0201381C
:10012000C0B2FF280AD118061B1A5B1853609360EF
:1001300080235B0211681942FCD070BD546094604A
:1001400016682E42FCD0EAE710E000E0FFFFFF0057
:10015000FEE700002549264870B581420AD0254BAC
:10016000C41E0022A34203D303331A1A920892003A
:10017000214B98472148224BC11E0022994203D8A7
:1001800003331A1A9208920000211E4B9847FF224F
:100190001D4B032193431D4A0C2593600222082422
:1001A00030261B4B1B485A62C3788B431343C370E2
:1001B000C378AB432343C370174B987BB04306000F
:1001C000202030439873987BA84304439C73987B0A
:1001D000884302439A738023104A51680B4353604B
:1001E0000F4B98470F4B9847FEE7C0463426000058
:1001F0000000002068000020452500006800002065
:100200004C060020572500000000000000ED00E033
:10021000FC70004100500041004800410040004196
:10022000FD240000D11B0000F0B517000A7885B04E
:1002300053060C0001909B0F012B52D16379097971
:100240002A4D1B020B432978994202D069789942C2
:1002500047D1E679A379360252B21E43002A0FDA5B
:100260000020012F0AD06378212B11D1072E3BD11A
:100270000300A91D320001981D4CA04705B0F0BD38
:100280001C4B984763780100202B03D0222B19D0F8
:100290000D2027E0072E27D1002F01D13B00E9E7F1
:1002A0003200154C02A8A0472B69002B05D107226C
:1002B000A81D02A9A0470020E0E702A8984700284F
:1002C000F5D1F8E700230A4E1A0019001800B047CC
:1002D0006B69002BEFD0E078A278000210439847BA
:1002E000E9E70A204042C9E70120FBE7840000203B
:1002F0005D2000008524000045250000F7B51500AD
:1003000001294FD0022900D176E0002900D075E004
:10031000836810681E00009302330193002802D105
:100320000A20404220E00821437982788B43022B47
:10033000F6D133789A4263D0FF2B63D1327069686B
:100340000522324B9847041E0FD1286804220378F7
:100350006968C0182D4B9847019B0136B342DDD127
:10036000012220002A4B5A71FEBD637922791B02BB
:10037000A778D2183800E178264B92B29847002827
:1003800042D17BB2244A002B09DAB770380090477B
:100390002C6020786968214B20189847D3E7009B90
:1003A0001F71F3E78468002A05D0136808225B797F
:1003B0009343022BB4D12378FF2B07D0FF25A078DD
:1003C0002570A84202D0164B9847A5706378FF2B82
:1003D00007D0FF25E0786570A84202D0104B9847FF
:1003E000E5702079FF2803D00D4B9847FF23237138
:1003F0000020074B5871B7E71B2092E70D2090E7CC
:1004000012208EE71C208CE714208AE7511600008A
:100410008400002061190000F11900006B16000033
:10042000C519000010B50A4B984701280CD8094897
:10043000094B0062C361094B1830984701200849F5
:10044000084B9847002010BD11204042FBE7C046F2
:100450009124000084000020FD0200002D240000F3
:1004600000000020A123000010B5074B0A005979B5
:100470000400002905D02100D878044C0123A047AE
:1004800010BD11204042FBE7840000205D200000E9
:100490000A0010B5032810D8094B02F01BF8020817
:1004A0000A0C18790221074B9847002010BDD87814
:1004B000F8E71961F9E75961F7E70D204042F5E7E0
:1004C00084000020851B0000014B58797047C0460E
:1004D0008400002000207047074B9A8C920604D5B8
:1004E0001022D9681142FCD004E0D021DA680A4019
:1004F000D02AFBD17047C04600080040002803D036
:10050000002901D00230C0B2142301305843014BFE
:10051000C0187047080100200F2370B50100807CCF
:10052000072503401A00CC7C083225405B01012DD1
:1005300008D01449520152181021D171124A9B1847
:10054000597270BD40252C4206D08026AC43CC7435
:100550000D4C1C196671A5710825CC7C5201AC4369
:10056000CC7400240949C9188C728C76054952183C
:100570006F21D171044A9B185972054B9B689847AB
:10058000DFE7C04600500041FF500041A8000020B6
:100590000801002020238B40DAB20F2310B504009D
:1005A000807C054903405B015B185A72034B0121B3
:1005B0001B69A268984710BDFF5000410801002048
:1005C00010B50300807CFF2809D04024DA7C224249
:1005D00005D0A243DA74024A14699A68A04710BD94
:1005E00008010020F7B59446837C134A01AE0D0044
:1005F0003280FF2B1AD04027C27C3A4216D00F22FD
:1006000013401C0008346201002910D00B4FD2198E
:10061000802717710949640164180949725D5B01FB
:100620005B18E27161465A72064B9847F7BD034961
:1006300052185771EEE7C046254A000000500041AD
:10064000FF500041C1050000F0B50D000F21837C73
:1006500085B00B409C46304B03AE338063465B0154
:100660000093634608332D495C01002D20D0095DBD
:100670004906490F009A2C01A418294A765D1419DD
:10068000A77AFFB2022917D101390F4214D0A77AF5
:10069000224A5B019B188F43009AA772DE71214B9F
:1006A0002940D218567204221F4B984705B0F0BD5E
:1006B0000C5D07212140DDE702213A000A4001924A
:1006C0000F4217D0A27AC77C8A43A272134A5B01F9
:1006D0009B18DE71009A134BD218072356723B40C9
:1006E000012BE3D17B06E1D5C17CC909A942DDD04C
:1006F0000022D9E7624651004D19094A2D015519CA
:10070000019A5B01AA72054A9B18DE71009A054B9B
:10071000D2185672CAE7C0460408000000500041D3
:10072000A8000020FF500041E50500008C2370B5B3
:10073000FF26094D9B00094CED1803212000084BB2
:1007400098470021A674E1741434AC42F5D16022BC
:10075000044B0548984770BD080100201C0100208B
:10076000C105000057250000A8000020F0B50F27A4
:1007700085B00191837C040002931F4000239942BD
:1007800005D04B4B7A019B185B699B049B0C258A17
:10079000484AAC46954202D06A1E12B294460722DD
:1007A000E07C02400392019A002A04D042497A0177
:1007B00052180221D171A26899186268A160914211
:1007C00040D22368521A59187B01394E92B20293D3
:1007D00083062CD52B1C954200D9131C9DB22A00F0
:1007E000364BE0689847324BE26879015B181A6132
:1007F0007B01F6187369AD049B0BAA0C9D0315438E
:10080000756173692E4A13407361019B002B08D1F7
:10081000039B4E22012B00D0043A2A497B015B182E
:100820009A72254A7B019B1880225A7139E08023F5
:10083000151C9B019A4200D91D1C7B01F318ADB217
:100840001961D5E710267A0130420ED0E37C1C49AD
:10085000B343E374164B9A18921953689B0B9B038E
:10086000536053680B405360CFE7039801281AD1B7
:10087000144812184B205072624613409D420CD10E
:100880004025E37C0298AB43E3740F4BDB68984749
:10089000002806D1E37C2B43E374002120000B4B9E
:1008A000984705B0F0BD074812184A20E3E7C04654
:1008B000A8000020FF030000005100414525000072
:1008C000FF3F00F0FF50004108010020C10500007B
:1008D0000F23F0B5857C85B004000E001D40039108
:1008E000019100290AD0614B6A019B1859680901DE
:1008F0008A0C0392596889048B0C0193238A009314
:10090000009A5B4B9A4203D01300013B9BB20093C9
:10091000019B009FE27C1F40072313400293002E9F
:1009200004D054496B015B180121D97193060FD58E
:100930006368002B0CD0A26821689B1A88181A1CC7
:100940009BB2BB4200D93A1CE1684B4B92B298472C
:1009500063686A019446002B2CD1E27CD10629D52C
:1009600030339A43103B1A43E2746246E1683F4BCE
:1009700042489950218A63445A688904090902400F
:100980000A435A605A68920B92035A60002E0BD1A8
:10099000029925226B01012903D1344AD218967697
:1009A0002D2237495B189A72324B6D01ED184023A6
:1009B0002B711DE0A168002E1CD0228ABA4219D9E1
:1009C0001022E37C9343E374019B5918A160029ABF
:1009D0006B01012A46D12A4A9B182D225A72002DFA
:1009E00002D1224BE2681A6000212000254B984773
:1009F00005B0F0BD039A5118A1608B42E7D92020C1
:100A0000E27C5B1A278A9BB2024216D0391C9F42B5
:100A100000D9191CE068154A8BB269015050134A7D
:100A20001648624451689B041B0901400B43536004
:100A300053689B0B9B035360A8E79F420BD2802017
:100A4000800183420CD8009A93432068074A4118DA
:100A500068011150E3E79F42F7D91043E074F4E7CF
:100A60000300F2E7064A9B182522B7E7A8000020FA
:100A7000FF0300000051004145250000FF3F00F04A
:100A8000FF500041C1050000802302009B000720A9
:100A90009A4214D8013BFF3B01389A420FD80138E3
:100AA000802A0CD80138402A09D80138202A06D8D3
:100AB0000138102A03D806309042804140427047E6
:100AC00010B52A4CA378DB0718D40323A2781A4266
:100AD000FCD10222237813420AD023789343237057
:100AE0000323A2781A42FCD10223A2781A42FCD135
:100AF000012323700233A2781A42FCD10123A27889
:100B00001A42FCD11A4B1B4A1A605A609A60DA608A
:100B10001A61194B98471F20184B1A68530B910CF8
:100B2000920103400140520F834200D105231F2947
:100B300000D10239072A00D1023A9B010B4312036C
:100B4000134323850323E2781A43E2700C22E178F1
:100B50000A43E27004222270A278100018401A4260
:100B6000FAD1074B63620123238110BD005000417D
:100B700008010020D50400002D070000246080003B
:100B8000A800002003220E4B9978114214D19978C5
:100B90001142FCD102221978C8B2114205D1024398
:100BA0001A70032299781142FCD180210020054A55
:100BB0001160054A1A83704711204042FBE7C04686
:100BC0000050004100E100E08D0200000121024AD6
:100BD00013898B43138170470050004180231843D1
:100BE000014B98727047C04600500041F7B50F2482
:100BF00004402E4B00910600C10947B2200001922B
:100C000098470321009B05000B400093022C44D819
:100C1000837CFF2B44D1009B002B10D1F943C9B238
:100C2000224B2000C9099847837CFF2B38D1F33B26
:100C300063431F4A9B58002B34D113202EE0002F12
:100C400014DA0C2262431A4B9B185A68002A19D1F5
:100C50000C236343164CE418636800200099EB6092
:100C6000019B01312B82E974AE74FEBD0C236343FA
:100C70000F4A9B58002B0BD00C2262430C4B9B1845
:100C80001B8900E05B89019A9A42D6DC002FDFDBEA
:100C90000C235C43064BE358DFE712204042E4E7B5
:100CA0001420FBE7002FE7DACBE7C046FD04000085
:100CB00068250000F7B50F2504000540022D1AD85D
:100CC00043B2C70901933900144B28009847837C2D
:100CD0000600FF2B0FD00322114B39009847072243
:100CE000F37C1340012B07D100220E4B0834640122
:100CF000E254FF237382F7BD63B2002B07DA702240
:100D0000094B6D01ED186B7893436B70F1E7064B5F
:100D10006401E418637893436370EAE7FD0400001C
:100D2000E505000000500041FF500041F7B50F24D9
:100D30000440C109474B45B220009847464B61012A
:100D4000CE1872780700D2B2022C00D97DE0837CE5
:100D50000193FF2B00D178E0404B5C18C37C072146
:100D60001800084001283BD1772311001940009159
:100D70001A4200D06CE0663B73703D8A384B280005
:100D80009847E023374ADB0500071840AB031340C0
:100D900003436360402180230F22AD04AD0C284340
:100DA0006061B1717371009B2C48A372A376019BA3
:100DB000AC031340FA685B011A50C01842682A4D10
:100DC0001540254345604268920B92034260224AD7
:100DD00000989B18B0225A71A03A99719A72FEBD80
:100DE000002D19DA702115000D400A4230D15B0741
:100DF0005B0E134373703F8A194B38009847E0230A
:100E00000007DB0518408023BF04BF0C3843606136
:100E10007371A5762800E2E715000D400A4217D14C
:100E20005B075B0F134373703F8A0D4B3800984785
:100E30000C4ABB031340E0220007D20510400343D5
:100E400063604023B371A572E4E712204042C6E715
:100E50001420FBE7FD040000FF500041A800002023
:100E6000890A000000C0FF0FFF3F00F0F8B507003F
:100E70000F26C40937400D0038002100294B984740
:100E80000200022F4AD8837C10203340A040012D5D
:100E900010D1254D5901C0B2491948712021A140F6
:100EA00022485B01C9B21B1899720823D17C0B43FD
:100EB000D37409E05B01002D29D11D495D181B4940
:100EC0005B18D979084201D100201CE02021A14003
:100ED000C0B25871C8B258721E7A314204D0012192
:100EE000A140C9B2187259710721D37C1940012958
:100EF0000AD1FF35EC792F31200008400C42E3D1B4
:100F000028398B43D374F8BD08218B43D0E7064AB8
:100F10009B189B791840431E9841F4E712204042E9
:100F2000F1E7C046FD04000000510041FF500041C0
:100F300000500041F8B50F231840114B44011B1914
:100F40000F0019685D68AD04AD0C022812D8002F9F
:100F500010D00C4BE4186378112B0ED11026227A96
:100F60000020324205D008223800074B984728005D
:100F70002672F8BD12204042FBE71320FBE7C04673
:100F8000A8000020FF50004145250000F0B50F25C6
:100F9000077A87B07BB23D40FF0939000293060013
:100FA0003A4B280098473A49038A04001A008B42BA
:100FB00001D05A1E92B271680A400192022D62D885
:100FC00080203268800582420DD3324D8818A842B5
:100FD00009D8032015000540024204D1029A002AD4
:100FE0000EDB994206D2E3680125002B08D11320BD
:100FF000404217E0019B002B16D0E368002B42D043
:10100000E37C02201B070DD4234B05A89847E17C05
:1010100040230A001A400392204A194206D005A82C
:101020009047012007B0F0BD019DE9E70B43E37451
:1010300005A890477F213368FA0123607368039FF6
:101040006360039BA360E37C0B40134369011D00B5
:1010500020239D430D43E574737A002B02D0019F3A
:101060007B425F411022E37C3F0193431F43029B7D
:1010700000212000E774002B03DA094B9847002079
:10108000D0E7084BFAE71220B2E7C046FD040000A3
:10109000FF030000FF7F0020A5240000B324000010
:1010A0006D070000D1080000002900D10549012882
:1010B00002D1054B596070470028FCD1024B1960E2
:1010C000F9E7C046D504000008010020002900D13E
:1010D0000749002802D1074B99607047012802D1C7
:1010E000044BD960F9E70228F7D1024B1961F4E704
:1010F000D504000008010020F7B56C4B1A8C91B2A2
:101100000191002A00D066E09A8B198B04200A40D6
:1011100011000140024204D09883654B1B68984738
:10112000F7BD80241600A400264022421DD0614A4B
:101130009A839A82923AFF3A1A835F4B1A8912076E
:10114000120F032A05D01A8D1207120F032A07D196
:101150000121002249015B1819891A814904490DAE
:101160000320534B5B689847DAE78024150025403D
:10117000224205D09C834E4B310005205B68F2E78C
:1011800070261400344032420AD04A4A9E839E821E
:101190001A834A4B9847464B290002205B68E2E7D6
:1011A0000825110029402A420CD0454A5470414A72
:1011B0009D839E821A83434B98473D4B210001201B
:1011C0005B68D0E7D20706D53A4A9A839A821E8393
:1011D000374B5B68C7E700260F2701253A4CA37CF5
:1011E000FF2B38D02A003B409A400199114232D05F
:1011F00036495A01521832495B015B181278997AC4
:101200000B001340114226D014217143284A521872
:1012100047211032D27D1140012911D1DA0603D5C0
:1012200020002B4B984716E0402219001140134232
:1012300001D0290001E09B060DD52000254B09E0D7
:1012400051B200291CDA5906F3D4190708D5290030
:101250002000214B9847013614341B2EBFD15FE785
:10126000990703D5290020001C4BF3E707210A400A
:10127000012AF0D100215A07EAD4DB06EBD5CFE7EB
:10128000202019000140034201D00021D5E7580772
:10129000DED42B4203D029002000114BDAE70721CE
:1012A0000A40012AD7D11A07E7D5D0E700500041FC
:1012B0000801002001020000A8000020D90400005D
:1012C000FF5000412D0700001C0100200751004184
:1012D0001905000095050000490600006D07000093
:1012E000D108000010B5024B1860024B984710BDA2
:1012F000F8030020FD000000044B10B51C68044BEF
:1013000098470100034B2000984710BDF8030020C8
:10131000B913000011010000064B1A7AD2B21A72FA
:101320005A7AD2B25A729A7AD2B29A72DA7AD2B21D
:10133000DA72704700040040064B10B55A685A60D4
:10134000054B9847054B9847054B9847FF20054BA1
:10135000984710BD004000411913000049140000D7
:1013600089140000FD1500000068002800D17047B6
:101370008842F9D10120FAE770B50C4B05000C004A
:1013800006689847012358404F22094B0949C0B2CB
:1013900098472B68002B02D12C60236070BD33006E
:1013A0003668002EFBD11C602660F7E76913000049
:1013B000C11300008C250000FA235B0158437047DD
:1013C000002800D100BE704701220020024B82B0ED
:1013D0001A7002B07047C046FC030020064810B5E2
:1013E000064B01309847064B9847064B06489847EE
:1013F000064B984710BDC046FC030020CD230000DB
:101400002504000045240000080000207924000085
:1014100010B5044B98470028FBD003200249034B2A
:10142000984710BDC9040000C913000091040000D2
:1014300010B5014B984710BDDD130000014B187823
:10144000C0B27047FC0300200D4B186A196A890F5F
:101450008A070C4901400A4302210A431A629A6929
:10146000114399611F211A7F0A401A771E39DA68E1
:10147000D2080A42FBD08022196A0A431A627047D6
:10148000000800400000FF0F02220121144B9A8443
:10149000DA6812090A42FBD0124ADA62FC22D2014F
:1014A0009A629B2252009A849A8C92080A4210D027
:1014B0001022D9681142FCD08022998C0A430A4933
:1014C0009A844A78D209FCD102219A698A439A61A6
:1014D00070470121DA6812090A42FBD0ECE7C046E6
:1014E0000008004080BB0104000C0040F8B5060075
:1014F0000D001400002804D0081E02D01000431E66
:101500009841F1221049114B9847370008373800AD
:101510000F4B98470028F8D000263800A95D0D4BE6
:10152000984738000A4B98470028FAD00136B44251
:10153000F3D80125002C00D025003800064B984731
:101540000028FAD02800F8BDAA250000C113000029
:10155000A71E0000991E0000B11E0000F7B505008F
:1015600014000191002804D0081E02D01000431E70
:10157000984186220C490D4B5200984700262F00B7
:10158000083738000A4B98470028F8D0094B380034
:101590009847019B98550136B442F0D80120002CA1
:1015A00000D02000FEBDC046AA250000C1130000E7
:1015B000BB1E00009F1E000070B504000D00002837
:1015C00002D00800431E98410749084B342298472F
:1015D00020002900064B08309847002803D1054B0E
:1015E0006360054B236070BDAA250000C113000095
:1015F0006D1E00005D150000ED140000C30709D545
:101600008023104A5B00936083235B02536053780E
:10161000DB09FCD1030708D504230A4AFF33936092
:10162000094B53605378DB09FCD1030608D5082326
:10163000044AFF339360054B53605378DB09FCD1B8
:101640007047C046000C004003030100070721005B
:1016500010B5884201D3002010BD0378012BFAD9C0
:1016600044789442F8D0C018F3E7884201D30020B0
:1016700070470378012BFAD94278042AF7D0052A5B
:10168000F6D0C018F1E7000070B50D4B150002222E
:101690000C00984700280FD170BD0378012B0DD99D
:1016A0004378022B0AD14379AB42F5D0C2788378D4
:1016B00012029B189BB2C018A042EED30020EBE7A9
:1016C0005116000070B50C0016000025A04201D391
:1016D000002070BD03222100054B98470028F8D058
:1016E0000378012BF4D9B542F3D0C0180135EDE7EA
:1016F0005116000002000F21002030B5094B1140A7
:101700005C7894420CD01D78002D01D18C4207D01A
:101710000130C4B2203340B20D2CF1D1012040423F
:1017200030BDC046400400200020704770B5084B13
:1017300004000D009847074B40011B189A780020C1
:10174000032A03D1290020009B69984770BDC04639
:10175000F516000040040020F0B5374B87B00F00AD
:10176000009001929847354D4401002F41D12E1928
:10177000F770295D002933D12200B4780C327078DB
:10178000F369AA18032C27D10C270131F757984782
:1017900003007078002B0BD0294B7380002F02DBE5
:1017A000863BFF3B18430121264B984707B0F0BD0D
:1017B00004220393B2700493002F0ADB80231843A2
:1017C00002AB1873012302AA537303A81E4B984758
:1017D000ECE70F231840F3E798470223B370E5E7DF
:1017E0000123B3702C19E178E369019A00989847B6
:1017F000DCE72B19012F0CD10222DA70295D0029B8
:1018000004D19A7000980F4B9847EBE705229A7025
:10181000E8E7022F08D10422DA702A5D002A01D1FC
:101820009F70C3E70122F2E7032F03D1A022D20069
:101830005A80D7E7054AFBE7F51600004004002070
:10184000050200006D0E00008D0F0000060600006E
:10185000F7B5184B0400984747013B00164D0C3371
:101860005B19190001932000144B98478026C0B2E1
:1018700026430096124E082806D001212000B047CA
:1018800001210098B047F7BDED1901270021200084
:10189000B04700210098B047200001996B69AF70F4
:1018A00098470028EFD1052339002000AB70B047DE
:1018B0003900E6E7F516000040040020350F00006F
:1018C0006D0E000070B5124B984700281EDBD02229
:1018D000104C00212000104B520098472300FF219C
:1018E0000D240E4A013CE4B259705A619A61DA61E2
:1018F0002033002CF6D10A4D20000A49A8470120C8
:101900000949A84702200949A847200070BDC046E0
:10191000C10A0000400400205725000029170000DC
:10192000CD100000511800002D17000059170000BD
:1019300010B5014B984710BDA910000010B5014B20
:10194000984710BD850B000010B5014B984710BD9E
:10195000CD0B000010B5014B984710BDDD0B00000A
:10196000F8B5104C06000D001700A047002813DA48
:10197000FF20A047041E12DB3A00290030000A4B6A
:101980009847002807DB03210020084B64011A193F
:101990000D405670E554F8BD14204042FBE7152079
:1019A000FBE7C046F5160000ED0B000040040020E8
:1019B000002110B502000800014B984710BDC04639
:1019C0006119000070B5074B05009847041E07DB3E
:1019D0002800054B9847FF230448640104196370ED
:1019E00070BDC046F5160000B50C00004004002094
:1019F00070B50C4B0400984700280FDB0A4D4001DE
:101A0000425D2D1851424A4101322000074BAA7015
:101A10009847002801DA0023AB7070BD12204042C5
:101A2000FBE7C046F5160000400400202D0D000025
:101A3000F0B5037A04008BB018000193324B98473D
:101A4000637A061E656802935BDB304B06A89847F5
:101A500073010093009A2E4B9E18B37804AAD71DE9
:101A60003B703A78D3B203932A4B012A1DD102323C
:101A7000B27006A89847264B009AD35C002B1FD063
:101A80000298019B421E9041D909C0B22368227A74
:101A900007930895002931D080231A4304AB1A75A7
:101AA00058751D4B07A8984708E006A898473B784B
:101AB0000120DAB2062B01D8184B98560BB0F0BDB6
:101AC000F27CB37C12029B189BB2002B05D104223E
:101AD00003981D000100B270D8E79D4200D91D0097
:101AE0000B4900208C46009A01006244127B7F2A39
:101AF000CCD99D429B4101315842C7E70F231A4080
:101B0000CCE712204042D9E7F5160000A5240000DA
:101B100040040020B32400008D0F0000C625000003
:101B2000F8B505000E1E1AD1124B9847041E1DDB96
:101B300002212800104FB84700280FD0310028009C
:101B4000B84700280ADB0D480D4B64012418638058
:101B5000320003212800E36998473000F8BD064BA6
:101B6000012900D0022128009847F7E712204042BF
:101B7000F4E7C046F51600006D0E0000400400209A
:101B80000103000070B50F4B14000D009847002CA6
:101B900000D10D4C002809DB012D08D0022D0BD0FF
:101BA000002D03D1094B40011818446170BD074B4B
:101BB000400118188461F9E7044B40011818C4610A
:101BC000F4E7C046F5160000291700004004002085
:101BD00013B50D4B98470D4B98470D4B98470D4B40
:101BE00098470028FBD0FA200B4BC00098470B4CBD
:101BF0000D220B490B4B200098470D2120000A4B6A
:101C000098470190FEE7C046C51E00003114000051
:101C1000111400003D140000F9120000E00500203E
:101C2000D4250000452500006904000030B50124DA
:101C30000C4BC5B2C0180378CAB2A3430A49234368
:101C400003706B085B180F201978254205D00140FE
:101C500012011143C9B2197030BD81430A431A7091
:101C6000FAE7C046404400413044004110B5162018
:101C7000034C0449A04717200349A04710BDC046A4
:101C80002D1C000002001600020017002023044A49
:101C9000116A0B431362034B034A5A807047C046D4
:101CA00000040040000C00401740000010B5054B38
:101CB000984700220449054B05489847054B98472B
:101CC00010BDC0468D1C000000140042B915000074
:101CD000200600206D1C000010B50248024B9847FA
:101CE00010BDC04610E000E0E5120000F8B5C025C8
:101CF00080238027114C124AED05FF055B04AB6081
:101D0000A762A262220004266B6158321378182061
:101D1000B34313700B490C4B984780230B4A9B0429
:101D2000AB60A762A2626B61593423781920B34378
:101D300023700749044B9847F8BDC0460044004152
:101D4000000100C0060018002D1C0000000200C0A9
:101D5000060019002022064BD9690A43DA614022A5
:101D600059690A435A61034B034A5A807047C04677
:101D700000040040000C00400647000010B5034B73
:101D80009847034B9847034B984710BD551D0000DB
:101D9000C5180000ED1C000010B5044B9847044B1B
:101DA0009847044B9847044B984710BD39130000DF
:101DB000AD1C0000D91C00007D1D0000C369194244
:101DC000FCD17047022210B50368032193430360DE
:101DD000014B984710BDC046BD1D00001B4B70B5A0
:101DE000C3189B0ADBB20400032B04D00020184A5E
:101DF0001849194B9847E369184DDB0711D402269F
:101E000003212000A8472368334205D02000144B4B
:101E1000984731002000A8470523032120002360B4
:101E2000A84720000121A8470E4B20002360032172
:101E3000A847C0239B02200063600721A847002019
:101E4000094BA381A0733034207070BD00F8FFBD32
:101E50003A020000E1250000C1130000BD1D000092
:101E6000C51D00000400104004C5FFFF70B505004B
:101E7000431E98410C00B4220449054BC0B2984758
:101E80002C602000034B984770BDC046E125000040
:101E9000C1130000DD1D0000036819857047036849
:101EA000188DC0B270470368187E01231840704730
:101EB0000368187E8007C00F70470368187E4007CC
:101EC000C00F704710B5024B9847024B984710BDA2
:101ED000991D000031140000064B10B51C69002C40
:101EE00000D110BD200063680022012198472468BA
:101EF000F5E7C0462C06002070B505000E00064B25
:101F0000DC68002C00D170BD6368002B02D031006A
:101F1000280098472468F4E72C060020F8B505004F
:101F20000E0017000B4B9C68002C01D12000F8BD5F
:101F30006368002B01D12468F6E73A0031002800DD
:101F40009847002804D00A30F5D001204042EEE73F
:101F50000120ECE72C060020054B10B55C68002C36
:101F600000D110BD6368002B00D098472468F6E7C5
:101F70002C06002010B51400002903D0012923D01D
:101F8000002010BD1378002BFAD15378052B0FD009
:101F9000092BF5D1E17892780E4B09021143D976DD
:101FA0004A1E91410331997601200B4B9847E7E790
:101FB0000A4B90789847E178A278090211434B1EAA
:101FC0009941044B0231EEE70A00054B2100002045
:101FD0009847D5E72C060020F91E0000551900008F
:101FE0001D1F000070B5002402260C4B98470C4DB5
:101FF00020006E830B4B6C7798470B4B287F9847DC
:102000000A4D210020000A4AA84731002000094A51
:10201000A8472000084B984770BDC046D91E000055
:102020002C060020C5190000B1190000851B000016
:1020300079200000751F0000F119000010B500287C
:1020400002D0012803D010BD024B9847FBE7024B9A
:102050009847F8E7F91E0000E51F00001FB502923F
:102060006A461073537301A8024B0191984705B05B
:1020700000BDC046311A0000F7B5B74B002204007E
:102080000D009847030000205A1C00D1C1E0013028
:10209000834200D1BDE02B781F221900914304D068
:1020A000802900D1B6E00020B3E0687801380A2822
:1020B000F9D800F005FA46F856F80BF8F8F806F8E3
:1020C0006000AA78002A0BD1A44B98470022012374
:1020D00011002000A24CA04743425841C0B298E0F2
:1020E000A04D2B6803CBA04B9847002800D190E06F
:1020F000C37881781B02C91889B2411804229B4B0E
:1021000001919847FF220090009B002BDED09E7823
:10211000964202D02F69002F0AD10098042203783A
:102120000199C0180090914B984732000090EBE75E
:102130006A46002138007B6898470028EDD03F6848
:10214000E9E7022BAFD1EE79AB7936021E43AAD173
:1021500031002879864B9847012332003100200056
:1021600054E0022B9FD1EB79AE791B021E439AD12A
:1021700001212879EEE7EC78AB7824021C432B7917
:102180006D79784E2D021D433368F27E03CB764B7A
:102190009847002887D004220090C37881781B02DA
:1021A000C91889B24118714F0191B847002800D170
:1021B00079E78378AB4210D1C378A3420DD1376958
:1021C0000090002F00D16EE701216A4638007B683D
:1021D0009847011E08D03F68F3E70098042203786F
:1021E0000199C0180090E0E76A4638007B6898477C
:1021F000002800D057E7002C04D00122AA40737FAA
:102200001343737700231A0019001800544CA04799
:102210000120FEBD68780A2800D944E700F064F97F
:10222000620043FF43FF43FF43FF43FF0B0043FFB5
:102230005A0043FF8300E978AB7809020B43090A8F
:10224000CAB2022917D0032A34D00020012AE0D1D3
:10225000AB79ED792D021D43424B1B6803CB434BF9
:102260009847011E00D11EE72A1C122D00D9122208
:10227000002392B22DE7AA79ED7901332D0215439F
:10228000384A1068167F03C8DAB2374B9847011EE8
:1022900000D108E7C37882781B02D21892B20023DB
:1022A000954205D9013E35406B425D41EBB21500C8
:1022B0002A000EE7AA79ED792D021543294A106804
:1022C000167F03C8DAB22B4B9847011E00D1EAE60D
:1022D0000278E4E72349CB7E4A69137049690023F9
:1022E00001223CE71F211E22180019401040134212
:1022F0000ED0022900D0D6E61D4B2879984703005E
:102300000020834200DA84E701300340009300E0BC
:102310000090144D02226946174B686998470023C4
:10232000022269691BE70F4E6B792979727F1B02C4
:102330000B431A4101241000204022421ED0346970
:10234000002C00D1AFE62A000221200063689847E4
:1023500000281BDA2468F3E71D1F0000D91E0000C7
:102360005D2000002C060020891600005116000098
:10237000211B0000C51600004525000073692200DE
:10238000187071690300054DA84741E77369012280
:10239000187000237169180038E7C0465D200000FE
:1023A00010B5012808D0022809D0002803D105481B
:1023B0000430054B984710BD02480830F9E7014842
:1023C0000C30F6E72C0600207913000070B50400ED
:1023D000431E98410C4A0D4B0D49C0B298470D4B16
:1023E000984700280EDB0C4D20220C4B00212800C2
:1023F000984700200A496C610A4CA04701200A490D
:10240000A047002070BDC04655030000C113000066
:10241000FC250000C51800002C06002057250000F0
:10242000591F0000311900003D20000010B50100C7
:102430000248034B1030984710BDC0462C060020C0
:102440007913000010B50A4B9C7E002C0BD100289C
:102450000CD002681860D2791A7701229A76054B5F
:102460009847200010BD04204042FBE70920FBE70D
:102470002C0600203D19000010B5014B984710BDF7
:1024800049190000014B58697047C0462C060020CE
:10249000034B987E1023184200D018007047C046A6
:1024A0002C060020EFF31083036072B6BFF35F8F3A
:1024B0007047BFF35F8F036883F310887047000095
:1024C00002B4714649084900095649008E4402BCCD
:1024D0007047C04602B4714649084900095C49008A
:1024E0008E4402BC7047C04603B4714649084000A0
:1024F0004900095E49008E4403BC704770B5002650
:102500000C4D0D4C641BA410A64209D1002600F00E
:1025100081F80A4D0A4C641BA410A64205D170BD77
:10252000B300EB5898470136EEE7B300EB589847F5
:102530000136F2E7202600002026000020260000B9
:1025400024260000002310B59A4200D110BDCC5CB7
:10255000C4540133F8E703008218934200D1704756
:1025600019700133F9E70000B803002000000000F3
:102570004000000078030020000000004000000040
:102580003803002000000000400000002E2E2F68BD
:10259000616C2F7574696C732F7372632F75746916
:1025A0006C735F6C6973742E63002E2E2F68616CE0
:1025B0002F7372632F68616C5F75736172745F73E0
:1025C000796E632E6300ED0101010102F0ED00015F
:1025D000010102F048656C6C6F20576F726C640AE1
:1025E000002E2E2F68706C2F736572636F6D2F68CD
:1025F000706C5F736572636F6D2E63002E2E2F7586
:1026000073622F6465766963652F75736264632EE8
:1026100063000000F8B5C046F8BC08BC9E46704791
:10262000DD000000F8B5C046F8BC08BC9E46704707
:04263000B5000000F1
:1026340000000000290200001000002065000020B6
:102644001201000202000040EB0304240001000018
:102654000001090243000201008032090400000164
:1026640002020000052400011005240101000424D5
:10267400020205240600010705820340000A09043A
:102684000100020A000000070501024000000705DE
:0826940081024000000000007B
:00000001FF
